 LuaMacro

 Timestamp is 54387416 (Sat Oct 11 04:04:38 2014)

 Preferred load address is 10000000

 Start         Length     Name                   Class
 0001:00000000 00000154H .idata$5                CODE
 0001:00000154 00000004H .CRT$XCA                CODE
 0001:00000158 00000004H .CRT$XCZ                CODE
 0001:0000015c 00000004H .CRT$XIA                CODE
 0001:00000160 0000000cH .CRT$XIC                CODE
 0001:0000016c 00000004H .CRT$XIZ                CODE
 0001:00000170 00000004H .CRT$XPA                CODE
 0001:00000174 00000004H .CRT$XPZ                CODE
 0001:00000178 00000004H .CRT$XTA                CODE
 0001:0000017c 00000004H .CRT$XTZ                CODE
 0001:00000180 00001ff0H .rdata                  CODE
 0001:00002170 0000000cH .rdata$sxdata           CODE
 0001:0000217c 00000004H .rtc$IAA                CODE
 0001:00002180 00000004H .rtc$IZZ                CODE
 0001:00002184 00000004H .rtc$TAA                CODE
 0001:00002188 00000004H .rtc$TZZ                CODE
 0001:00002190 00005002H .text                   CODE
 0001:00007198 000001ecH .xdata$x                CODE
 0001:00007384 0000003cH .idata$2                CODE
 0001:000073c0 00000014H .idata$3                CODE
 0001:000073d4 00000154H .idata$4                CODE
 0001:00007528 00000618H .idata$6                CODE
 0001:00007b40 0000019cH .edata                  CODE
 0002:00000000 00000b50H .data                   DATA
 0002:00000b60 00001780H .bss                    DATA
 0003:00000000 00000058H .rsrc$01                DATA
 0003:00000060 00000370H .rsrc$02                DATA

  Address         Publics by Value              Rva+Base       Lib:Object

 0000:00000000       __except_list              00000000     <absolute>
 0000:00000003       ___safe_se_handler_count   00000003     <absolute>
 0000:00000000       ___ImageBase               10000000     <linker-defined>
 0001:00000000       __imp__DeleteCriticalSection@4 10001000     kernel32:KERNEL32.dll
 0001:00000004       __imp__GetModuleFileNameW@12 10001004     kernel32:KERNEL32.dll
 0001:00000008       __imp__InitializeCriticalSection@4 10001008     kernel32:KERNEL32.dll
 0001:0000000c       __imp__LeaveCriticalSection@4 1000100c     kernel32:KERNEL32.dll
 0001:00000010       __imp__EnterCriticalSection@4 10001010     kernel32:KERNEL32.dll
 0001:00000014       __imp__GetModuleHandleW@4  10001014     kernel32:KERNEL32.dll
 0001:00000018       __imp__SetLastError@4      10001018     kernel32:KERNEL32.dll
 0001:0000001c       __imp__GetProcAddress@8    1000101c     kernel32:KERNEL32.dll
 0001:00000020       __imp__GetStringTypeW@16   10001020     kernel32:KERNEL32.dll
 0001:00000024       __imp__MultiByteToWideChar@24 10001024     kernel32:KERNEL32.dll
 0001:00000028       __imp__LCMapStringW@24     10001028     kernel32:KERNEL32.dll
 0001:0000002c       __imp__LoadLibraryW@4      1000102c     kernel32:KERNEL32.dll
 0001:00000030       __imp__HeapReAlloc@16      10001030     kernel32:KERNEL32.dll
 0001:00000034       __imp__HeapAlloc@12        10001034     kernel32:KERNEL32.dll
 0001:00000038       __imp__IsProcessorFeaturePresent@4 10001038     kernel32:KERNEL32.dll
 0001:0000003c       __imp__RtlUnwind@16        1000103c     kernel32:KERNEL32.dll
 0001:00000040       __imp__IsValidCodePage@4   10001040     kernel32:KERNEL32.dll
 0001:00000044       __imp__GetOEMCP@0          10001044     kernel32:KERNEL32.dll
 0001:00000048       __imp__GetACP@0            10001048     kernel32:KERNEL32.dll
 0001:0000004c       __imp__GetCPInfo@8         1000104c     kernel32:KERNEL32.dll
 0001:00000050       __imp__WriteFile@20        10001050     kernel32:KERNEL32.dll
 0001:00000054       __imp__GetSystemTimeAsFileTime@4 10001054     kernel32:KERNEL32.dll
 0001:00000058       __imp__GetCurrentProcessId@0 10001058     kernel32:KERNEL32.dll
 0001:0000005c       __imp__GetTickCount@0      1000105c     kernel32:KERNEL32.dll
 0001:00000060       __imp__QueryPerformanceCounter@4 10001060     kernel32:KERNEL32.dll
 0001:00000064       __imp__HeapDestroy@4       10001064     kernel32:KERNEL32.dll
 0001:00000068       __imp__HeapCreate@12       10001068     kernel32:KERNEL32.dll
 0001:0000006c       __imp__GetEnvironmentStringsW@0 1000106c     kernel32:KERNEL32.dll
 0001:00000070       __imp__WideCharToMultiByte@32 10001070     kernel32:KERNEL32.dll
 0001:00000074       __imp__FreeEnvironmentStringsW@4 10001074     kernel32:KERNEL32.dll
 0001:00000078       __imp__GetModuleFileNameA@12 10001078     kernel32:KERNEL32.dll
 0001:0000007c       __imp__GetStartupInfoW@4   1000107c     kernel32:KERNEL32.dll
 0001:00000080       __imp__GetFileType@4       10001080     kernel32:KERNEL32.dll
 0001:00000084       __imp__GetStdHandle@4      10001084     kernel32:KERNEL32.dll
 0001:00000088       __imp__GetLastError@0      10001088     kernel32:KERNEL32.dll
 0001:0000008c       __imp__SetConsoleCtrlHandler@8 1000108c     kernel32:KERNEL32.dll
 0001:00000090       __imp__GetCurrentThreadId@0 10001090     kernel32:KERNEL32.dll
 0001:00000094       __imp__GetCommandLineA@0   10001094     kernel32:KERNEL32.dll
 0001:00000098       __imp__InitializeCriticalSectionAndSpinCount@8 10001098     kernel32:KERNEL32.dll
 0001:0000009c       __imp__TlsAlloc@0          1000109c     kernel32:KERNEL32.dll
 0001:000000a0       __imp__TlsGetValue@4       100010a0     kernel32:KERNEL32.dll
 0001:000000a4       __imp__TlsSetValue@8       100010a4     kernel32:KERNEL32.dll
 0001:000000a8       __imp__TlsFree@4           100010a8     kernel32:KERNEL32.dll
 0001:000000ac       __imp__InterlockedIncrement@4 100010ac     kernel32:KERNEL32.dll
 0001:000000b0       __imp__InterlockedDecrement@4 100010b0     kernel32:KERNEL32.dll
 0001:000000b4       __imp__UnhandledExceptionFilter@4 100010b4     kernel32:KERNEL32.dll
 0001:000000b8       __imp__SetUnhandledExceptionFilter@4 100010b8     kernel32:KERNEL32.dll
 0001:000000bc       __imp__IsDebuggerPresent@0 100010bc     kernel32:KERNEL32.dll
 0001:000000c0       __imp__TerminateProcess@8  100010c0     kernel32:KERNEL32.dll
 0001:000000c4       __imp__GetCurrentProcess@0 100010c4     kernel32:KERNEL32.dll
 0001:000000c8       __imp__Sleep@4             100010c8     kernel32:KERNEL32.dll
 0001:000000cc       __imp__ExitProcess@4       100010cc     kernel32:KERNEL32.dll
 0001:000000d0       __imp__HeapFree@12         100010d0     kernel32:KERNEL32.dll
 0001:000000d4       __imp__SetHandleCount@4    100010d4     kernel32:KERNEL32.dll
 0001:000000d8       __imp__HeapSize@12         100010d8     kernel32:KERNEL32.dll
 0001:000000dc       \177KERNEL32_NULL_THUNK_DATA 100010dc     kernel32:KERNEL32.dll
 0001:000000e0       __imp__lua_sethook         100010e0     lua51:lua51.dll
 0001:000000e4       __imp__lua_close           100010e4     lua51:lua51.dll
 0001:000000e8       __imp__luaL_newstate       100010e8     lua51:lua51.dll
 0001:000000ec       __imp__luaL_ref            100010ec     lua51:lua51.dll
 0001:000000f0       __imp__lua_newuserdata     100010f0     lua51:lua51.dll
 0001:000000f4       __imp__lua_setfield        100010f4     lua51:lua51.dll
 0001:000000f8       __imp__lua_pushcclosure    100010f8     lua51:lua51.dll
 0001:000000fc       __imp__lua_settop          100010fc     lua51:lua51.dll
 0001:00000100       __imp__lua_pushboolean     10001100     lua51:lua51.dll
 0001:00000104       __imp__lua_toboolean       10001104     lua51:lua51.dll
 0001:00000108       __imp__lua_getfield        10001108     lua51:lua51.dll
 0001:0000010c       __imp__luaL_error          1000110c     lua51:lua51.dll
 0001:00000110       \177lua51_NULL_THUNK_DATA  10001110     lua51:lua51.dll
 0001:00000114       __imp__LF_ProcessEnvVars   10001114     luafar3:luafar3.dll
 0001:00000118       __imp__LF_DlgProc          10001118     luafar3:luafar3.dll
 0001:0000011c       __imp__LF_InitLuaState2    1000111c     luafar3:luafar3.dll
 0001:00000120       __imp__LF_GetGlobalInfo    10001120     luafar3:luafar3.dll
 0001:00000124       __imp__LF_RunDefaultScript 10001124     luafar3:luafar3.dll
 0001:00000128       __imp__LF_GetPluginInfo    10001128     luafar3:luafar3.dll
 0001:0000012c       __imp__LF_ProcessSynchroEvent 1000112c     luafar3:luafar3.dll
 0001:00000130       __imp__LF_ExitFAR          10001130     luafar3:luafar3.dll
 0001:00000134       __imp__LF_Open             10001134     luafar3:luafar3.dll
 0001:00000138       __imp__LF_Configure        10001138     luafar3:luafar3.dll
 0001:0000013c       __imp__LF_ProcessEditorInput 1000113c     luafar3:luafar3.dll
 0001:00000140       __imp__LF_ProcessEditorEvent 10001140     luafar3:luafar3.dll
 0001:00000144       __imp__LF_ProcessViewerEvent 10001144     luafar3:luafar3.dll
 0001:00000148       __imp__LF_ProcessDialogEvent 10001148     luafar3:luafar3.dll
 0001:0000014c       __imp__LF_InitLuaState1    1000114c     luafar3:luafar3.dll
 0001:00000150       \177luafar3_NULL_THUNK_DATA 10001150     luafar3:luafar3.dll
 0001:00000154       ___xc_a                    10001154     LIBCMT:crt0init.obj
 0001:00000158       ___xc_z                    10001158     LIBCMT:crt0init.obj
 0001:0000015c       ___xi_a                    1000115c     LIBCMT:crt0init.obj
 0001:0000016c       ___xi_z                    1000116c     LIBCMT:crt0init.obj
 0001:00000170       ___xp_a                    10001170     LIBCMT:crt0init.obj
 0001:00000174       ___xp_z                    10001174     LIBCMT:crt0init.obj
 0001:00000178       ___xt_a                    10001178     LIBCMT:crt0init.obj
 0001:0000017c       ___xt_z                    1000117c     LIBCMT:crt0init.obj
 0001:00000998       ??_C@_0N@IHACIAEK@interrupted?$CB?$AA@ 10001998     luaplug.obj
 0001:000009a8       ??_C@_08LOAFAMNO@_luaplug?$AA@ 100019a8     luaplug.obj
 0001:000009b4       ??_C@_1O@NKFKHEOM@?$AAL?$AAU?$AAA?$AAF?$AAA?$AAR?$AA?$AA@ 100019b4     luaplug.obj
 0001:000009c4       ??_C@_0BE@CHABKMMA@IsLuaStateRecreated?$AA@ 100019c4     luaplug.obj
 0001:000009d8       ??_C@_0BB@NFAIBGGI@RecreateLuaState?$AA@ 100019d8     luaplug.obj
 0001:000009f0       __imp__EncodePointer@4     100019f0     vc_crt_fix.obj
 0001:000009f4       __imp__DecodePointer@4     100019f4     vc_crt_fix.obj
 0001:000009f8       __imp__GetModuleHandleExW@12 100019f8     vc_crt_fix.obj
 0001:00000a10       ??_C@_0O@NLDKAIKN@EncodePointer?$AA@ 10001a10     vc_crt_fix_impl.obj
 0001:00000a20       ??_C@_0O@KBPMFGHI@DecodePointer?$AA@ 10001a20     vc_crt_fix_impl.obj
 0001:00000a30       ??_C@_0BD@GIGEJCNH@GetModuleHandleExW?$AA@ 10001a30     vc_crt_fix_impl.obj
 0001:00000a44       __pRawDllMain              10001a44     LIBCMT:dllcrt0.obj
 0001:00000a44       __pDefaultRawDllMain       10001a44     LIBCMT:dllcrt0.obj
 0001:00000a48       ??_C@_1BK@DBDEIDLH@?$AAK?$AAE?$AAR?$AAN?$AAE?$AAL?$AA3?$AA2?$AA?4?$AAD?$AAL?$AAL?$AA?$AA@ 10001a48     LIBCMT:tidtable.obj
 0001:00000a64       ??_C@_07PEJMOBNF@FlsFree?$AA@ 10001a64     LIBCMT:tidtable.obj
 0001:00000a6c       ??_C@_0M@JCPCPOEF@FlsSetValue?$AA@ 10001a6c     LIBCMT:tidtable.obj
 0001:00000a78       ??_C@_0M@GDNOONDI@FlsGetValue?$AA@ 10001a78     LIBCMT:tidtable.obj
 0001:00000a84       ??_C@_08KNHFBNJ@FlsAlloc?$AA@ 10001a84     LIBCMT:tidtable.obj
 0001:00000a90       __XcptActTab               10001a90     LIBCMT:winxfltr.obj
 0001:00000b20       __First_FPE_Indx           10001b20     LIBCMT:winxfltr.obj
 0001:00000b24       __Num_FPE                  10001b24     LIBCMT:winxfltr.obj
 0001:00000b28       __XcptActTabSize           10001b28     LIBCMT:winxfltr.obj
 0001:00000b2c       __XcptActTabCount          10001b2c     LIBCMT:winxfltr.obj
 0001:00000b30       ??_C@_0P@MIGLKIOC@CorExitProcess?$AA@ 10001b30     LIBCMT:crt0dat.obj
 0001:00000b40       ??_C@_1BI@BGOHAHKC@?$AAm?$AAs?$AAc?$AAo?$AAr?$AAe?$AAe?$AA?4?$AAd?$AAl?$AAl?$AA?$AA@ 10001b40     LIBCMT:crt0dat.obj
 0001:00000b58       ??_C@_1BO@BKOMIGKJ@?$AAr?$AAu?$AAn?$AAt?$AAi?$AAm?$AAe?$AA?5?$AAe?$AAr?$AAr?$AAo?$AAr?$AA?5?$AA?$AA@ 10001b58     LIBCMT:crt0msg.obj
 0001:00000b78       ??_C@_15JNBOKNOG@?$AA?$AN?$AA?6?$AA?$AA@ 10001b78     LIBCMT:crt0msg.obj
 0001:00000b80       ??_C@_1BM@JBBEPPHI@?$AAT?$AAL?$AAO?$AAS?$AAS?$AA?5?$AAe?$AAr?$AAr?$AAo?$AAr?$AA?$AN?$AA?6?$AA?$AA@ 10001b80     LIBCMT:crt0msg.obj
 0001:00000b9c       ??_C@_1BK@KMOMNAAI@?$AAS?$AAI?$AAN?$AAG?$AA?5?$AAe?$AAr?$AAr?$AAo?$AAr?$AA?$AN?$AA?6?$AA?$AA@ 10001b9c     LIBCMT:crt0msg.obj
 0001:00000bb8       ??_C@_1BO@BFCDCGC@?$AAD?$AAO?$AAM?$AAA?$AAI?$AAN?$AA?5?$AAe?$AAr?$AAr?$AAo?$AAr?$AA?$AN?$AA?6?$AA?$AA@ 10001bb8     LIBCMT:crt0msg.obj
 0001:00000bd8       ??_C@_1BOO@KGEDBGAJ@?$AAR?$AA6?$AA0?$AA3?$AA3?$AA?$AN?$AA?6?$AA?9?$AA?5?$AAA?$AAt?$AAt?$AAe?$AAm?$AAp?$AAt?$AA?5?$AAt?$AAo?$AA?5?$AAu?$AAs?$AAe?$AA?5?$AAM?$AAS?$AAI?$AAL?$AA?5?$AAc?$AAo?$AAd@ 10001bd8     LIBCMT:crt0msg.obj
 0001:00000dc8       ??_C@_1GG@GOPILAJP@?$AAR?$AA6?$AA0?$AA3?$AA2?$AA?$AN?$AA?6?$AA?9?$AA?5?$AAn?$AAo?$AAt?$AA?5?$AAe?$AAn?$AAo?$AAu?$AAg?$AAh?$AA?5?$AAs?$AAp?$AAa?$AAc?$AAe?$AA?5?$AAf?$AAo?$AAr?$AA?5?$AAl?$AAo@ 10001dc8     LIBCMT:crt0msg.obj
 0001:00000e30       ??_C@_1MG@ENCOOIDF@?$AAR?$AA6?$AA0?$AA3?$AA1?$AA?$AN?$AA?6?$AA?9?$AA?5?$AAA?$AAt?$AAt?$AAe?$AAm?$AAp?$AAt?$AA?5?$AAt?$AAo?$AA?5?$AAi?$AAn?$AAi?$AAt?$AAi?$AAa?$AAl?$AAi?$AAz?$AAe?$AA?5?$AAt@ 10001e30     LIBCMT:crt0msg.obj
 0001:00000ef8       ??_C@_1DO@BMFCDCD@?$AAR?$AA6?$AA0?$AA3?$AA0?$AA?$AN?$AA?6?$AA?9?$AA?5?$AAC?$AAR?$AAT?$AA?5?$AAn?$AAo?$AAt?$AA?5?$AAi?$AAn?$AAi?$AAt?$AAi?$AAa?$AAl?$AAi?$AAz?$AAe?$AAd?$AA?$AN?$AA?6?$AA?$AA@ 10001ef8     LIBCMT:crt0msg.obj
 0001:00000f38       ??_C@_1EK@HHFLMAOL@?$AAR?$AA6?$AA0?$AA2?$AA8?$AA?$AN?$AA?6?$AA?9?$AA?5?$AAu?$AAn?$AAa?$AAb?$AAl?$AAe?$AA?5?$AAt?$AAo?$AA?5?$AAi?$AAn?$AAi?$AAt?$AAi?$AAa?$AAl?$AAi?$AAz?$AAe?$AA?5?$AAh?$AAe@ 10001f38     LIBCMT:crt0msg.obj
 0001:00000f88       ??_C@_1GK@MFGOKLAG@?$AAR?$AA6?$AA0?$AA2?$AA7?$AA?$AN?$AA?6?$AA?9?$AA?5?$AAn?$AAo?$AAt?$AA?5?$AAe?$AAn?$AAo?$AAu?$AAg?$AAh?$AA?5?$AAs?$AAp?$AAa?$AAc?$AAe?$AA?5?$AAf?$AAo?$AAr?$AA?5?$AAl?$AAo@ 10001f88     LIBCMT:crt0msg.obj
 0001:00000ff8       ??_C@_1GK@MCAAGJMO@?$AAR?$AA6?$AA0?$AA2?$AA6?$AA?$AN?$AA?6?$AA?9?$AA?5?$AAn?$AAo?$AAt?$AA?5?$AAe?$AAn?$AAo?$AAu?$AAg?$AAh?$AA?5?$AAs?$AAp?$AAa?$AAc?$AAe?$AA?5?$AAf?$AAo?$AAr?$AA?5?$AAs?$AAt@ 10001ff8     LIBCMT:crt0msg.obj
 0001:00001068       ??_C@_1EM@MAADIHMB@?$AAR?$AA6?$AA0?$AA2?$AA5?$AA?$AN?$AA?6?$AA?9?$AA?5?$AAp?$AAu?$AAr?$AAe?$AA?5?$AAv?$AAi?$AAr?$AAt?$AAu?$AAa?$AAl?$AA?5?$AAf?$AAu?$AAn?$AAc?$AAt?$AAi?$AAo?$AAn?$AA?5?$AAc@ 10002068     LIBCMT:crt0msg.obj
 0001:000010b8       ??_C@_1GK@FHCKBEFA@?$AAR?$AA6?$AA0?$AA2?$AA4?$AA?$AN?$AA?6?$AA?9?$AA?5?$AAn?$AAo?$AAt?$AA?5?$AAe?$AAn?$AAo?$AAu?$AAg?$AAh?$AA?5?$AAs?$AAp?$AAa?$AAc?$AAe?$AA?5?$AAf?$AAo?$AAr?$AA?5?$AA_?$AAo@ 100020b8     LIBCMT:crt0msg.obj
 0001:00001128       ??_C@_1FC@ECHBIFBC@?$AAR?$AA6?$AA0?$AA1?$AA9?$AA?$AN?$AA?6?$AA?9?$AA?5?$AAu?$AAn?$AAa?$AAb?$AAl?$AAe?$AA?5?$AAt?$AAo?$AA?5?$AAo?$AAp?$AAe?$AAn?$AA?5?$AAc?$AAo?$AAn?$AAs?$AAo?$AAl?$AAe?$AA?5@ 10002128     LIBCMT:crt0msg.obj
 0001:00001180       ??_C@_1EC@JIBHAOPH@?$AAR?$AA6?$AA0?$AA1?$AA8?$AA?$AN?$AA?6?$AA?9?$AA?5?$AAu?$AAn?$AAe?$AAx?$AAp?$AAe?$AAc?$AAt?$AAe?$AAd?$AA?5?$AAh?$AAe?$AAa?$AAp?$AA?5?$AAe?$AAr?$AAr?$AAo?$AAr?$AA?$AN?$AA?6@ 10002180     LIBCMT:crt0msg.obj
 0001:000011c8       ??_C@_1FK@BEOGODMC@?$AAR?$AA6?$AA0?$AA1?$AA7?$AA?$AN?$AA?6?$AA?9?$AA?5?$AAu?$AAn?$AAe?$AAx?$AAp?$AAe?$AAc?$AAt?$AAe?$AAd?$AA?5?$AAm?$AAu?$AAl?$AAt?$AAi?$AAt?$AAh?$AAr?$AAe?$AAa?$AAd?$AA?5@ 100021c8     LIBCMT:crt0msg.obj
 0001:00001228       ??_C@_1FI@LOGNIKDM@?$AAR?$AA6?$AA0?$AA1?$AA6?$AA?$AN?$AA?6?$AA?9?$AA?5?$AAn?$AAo?$AAt?$AA?5?$AAe?$AAn?$AAo?$AAu?$AAg?$AAh?$AA?5?$AAs?$AAp?$AAa?$AAc?$AAe?$AA?5?$AAf?$AAo?$AAr?$AA?5?$AAt?$AAh@ 10002228     LIBCMT:crt0msg.obj
 0001:00001280       ??_C@_1EG@BEHAGFJD@?$AAR?$AA6?$AA0?$AA1?$AA0?$AA?$AN?$AA?6?$AA?9?$AA?5?$AAa?$AAb?$AAo?$AAr?$AAt?$AA?$CI?$AA?$CJ?$AA?5?$AAh?$AAa?$AAs?$AA?5?$AAb?$AAe?$AAe?$AAn?$AA?5?$AAc?$AAa?$AAl?$AAl?$AAe?$AAd@ 10002280     LIBCMT:crt0msg.obj
 0001:000012c8       ??_C@_1FI@HONFMGBI@?$AAR?$AA6?$AA0?$AA0?$AA9?$AA?$AN?$AA?6?$AA?9?$AA?5?$AAn?$AAo?$AAt?$AA?5?$AAe?$AAn?$AAo?$AAu?$AAg?$AAh?$AA?5?$AAs?$AAp?$AAa?$AAc?$AAe?$AA?5?$AAf?$AAo?$AAr?$AA?5?$AAe?$AAn@ 100022c8     LIBCMT:crt0msg.obj
 0001:00001320       ??_C@_1FE@LLNEDJMD@?$AAR?$AA6?$AA0?$AA0?$AA8?$AA?$AN?$AA?6?$AA?9?$AA?5?$AAn?$AAo?$AAt?$AA?5?$AAe?$AAn?$AAo?$AAu?$AAg?$AAh?$AA?5?$AAs?$AAp?$AAa?$AAc?$AAe?$AA?5?$AAf?$AAo?$AAr?$AA?5?$AAa?$AAr@ 10002320     LIBCMT:crt0msg.obj
 0001:00001378       ??_C@_1FK@PGACCAFB@?$AAR?$AA6?$AA0?$AA0?$AA2?$AA?$AN?$AA?6?$AA?9?$AA?5?$AAf?$AAl?$AAo?$AAa?$AAt?$AAi?$AAn?$AAg?$AA?5?$AAp?$AAo?$AAi?$AAn?$AAt?$AA?5?$AAs?$AAu?$AAp?$AAp?$AAo?$AAr?$AAt?$AA?5@ 10002378     LIBCMT:crt0msg.obj
 0001:00001488       ??_C@_1EK@MBDPDCGA@?$AAM?$AAi?$AAc?$AAr?$AAo?$AAs?$AAo?$AAf?$AAt?$AA?5?$AAV?$AAi?$AAs?$AAu?$AAa?$AAl?$AA?5?$AAC?$AA?$CL?$AA?$CL?$AA?5?$AAR?$AAu?$AAn?$AAt?$AAi?$AAm?$AAe?$AA?5?$AAL?$AAi?$AAb@ 10002488     LIBCMT:crt0msg.obj
 0001:000014d4       ??_C@_15IABLJNFO@?$AA?6?$AA?6?$AA?$AA@ 100024d4     LIBCMT:crt0msg.obj
 0001:000014dc       ??_C@_17LGKOMLJ@?$AA?4?$AA?4?$AA?4?$AA?$AA@ 100024dc     LIBCMT:crt0msg.obj
 0001:000014e4       ??_C@_1CO@EAEJAADC@?$AA?$DM?$AAp?$AAr?$AAo?$AAg?$AAr?$AAa?$AAm?$AA?5?$AAn?$AAa?$AAm?$AAe?$AA?5?$AAu?$AAn?$AAk?$AAn?$AAo?$AAw?$AAn?$AA?$DO?$AA?$AA@ 100024e4     LIBCMT:crt0msg.obj
 0001:00001514       ??_C@_1DE@JNGNBFGO@?$AAR?$AAu?$AAn?$AAt?$AAi?$AAm?$AAe?$AA?5?$AAE?$AAr?$AAr?$AAo?$AAr?$AA?$CB?$AA?6?$AA?6?$AAP?$AAr?$AAo?$AAg?$AAr?$AAa?$AAm?$AA?3?$AA?5?$AA?$AA@ 10002514     LIBCMT:crt0msg.obj
 0001:00001548       ??_C@_1BC@GDGBMEMK@?$AAH?$AAH?$AA?3?$AAm?$AAm?$AA?3?$AAs?$AAs?$AA?$AA@ 10002548     LIBCMT:nlsdata2.obj
 0001:0000155c       ??_C@_1CI@KNAKOEBC@?$AAd?$AAd?$AAd?$AAd?$AA?0?$AA?5?$AAM?$AAM?$AAM?$AAM?$AA?5?$AAd?$AAd?$AA?0?$AA?5?$AAy?$AAy?$AAy?$AAy?$AA?$AA@ 1000255c     LIBCMT:nlsdata2.obj
 0001:00001584       ??_C@_1BC@IEBCMHCM@?$AAM?$AAM?$AA?1?$AAd?$AAd?$AA?1?$AAy?$AAy?$AA?$AA@ 10002584     LIBCMT:nlsdata2.obj
 0001:00001598       ??_C@_15CLMNNGEL@?$AAP?$AAM?$AA?$AA@ 10002598     LIBCMT:nlsdata2.obj
 0001:000015a0       ??_C@_15ODEHAHHF@?$AAA?$AAM?$AA?$AA@ 100025a0     LIBCMT:nlsdata2.obj
 0001:000015a8       ??_C@_1BC@FEMKIFH@?$AAD?$AAe?$AAc?$AAe?$AAm?$AAb?$AAe?$AAr?$AA?$AA@ 100025a8     LIBCMT:nlsdata2.obj
 0001:000015bc       ??_C@_1BC@BGLIFPF@?$AAN?$AAo?$AAv?$AAe?$AAm?$AAb?$AAe?$AAr?$AA?$AA@ 100025bc     LIBCMT:nlsdata2.obj
 0001:000015d0       ??_C@_1BA@EPANDLNG@?$AAO?$AAc?$AAt?$AAo?$AAb?$AAe?$AAr?$AA?$AA@ 100025d0     LIBCMT:nlsdata2.obj
 0001:000015e0       ??_C@_1BE@DKAAMBJL@?$AAS?$AAe?$AAp?$AAt?$AAe?$AAm?$AAb?$AAe?$AAr?$AA?$AA@ 100025e0     LIBCMT:nlsdata2.obj
 0001:000015f4       ??_C@_1O@PAHLKOAC@?$AAA?$AAu?$AAg?$AAu?$AAs?$AAt?$AA?$AA@ 100025f4     LIBCMT:nlsdata2.obj
 0001:00001604       ??_C@_19BIFMLPCD@?$AAJ?$AAu?$AAl?$AAy?$AA?$AA@ 10002604     LIBCMT:nlsdata2.obj
 0001:00001610       ??_C@_19EPFLPGAP@?$AAJ?$AAu?$AAn?$AAe?$AA?$AA@ 10002610     LIBCMT:nlsdata2.obj
 0001:0000161c       ??_C@_1M@GJNLMHFD@?$AAA?$AAp?$AAr?$AAi?$AAl?$AA?$AA@ 1000261c     LIBCMT:nlsdata2.obj
 0001:00001628       ??_C@_1M@IKEENEDF@?$AAM?$AAa?$AAr?$AAc?$AAh?$AA?$AA@ 10002628     LIBCMT:nlsdata2.obj
 0001:00001634       ??_C@_1BC@JGDDFFAM@?$AAF?$AAe?$AAb?$AAr?$AAu?$AAa?$AAr?$AAy?$AA?$AA@ 10002634     LIBCMT:nlsdata2.obj
 0001:00001648       ??_C@_1BA@EFMEIEBA@?$AAJ?$AAa?$AAn?$AAu?$AAa?$AAr?$AAy?$AA?$AA@ 10002648     LIBCMT:nlsdata2.obj
 0001:00001658       ??_C@_17EGKACKIF@?$AAD?$AAe?$AAc?$AA?$AA@ 10002658     LIBCMT:nlsdata2.obj
 0001:00001660       ??_C@_17BBDMLCIG@?$AAN?$AAo?$AAv?$AA?$AA@ 10002660     LIBCMT:nlsdata2.obj
 0001:00001668       ??_C@_17FNLKOI@?$AAO?$AAc?$AAt?$AA?$AA@ 10002668     LIBCMT:nlsdata2.obj
 0001:00001670       ??_C@_17HCHCOKMG@?$AAS?$AAe?$AAp?$AA?$AA@ 10002670     LIBCMT:nlsdata2.obj
 0001:00001678       ??_C@_17ICPELBCN@?$AAA?$AAu?$AAg?$AA?$AA@ 10002678     LIBCMT:nlsdata2.obj
 0001:00001680       ??_C@_17IJPCKHK@?$AAJ?$AAu?$AAl?$AA?$AA@ 10002680     LIBCMT:nlsdata2.obj
 0001:00001688       ??_C@_17KCJGOCPB@?$AAJ?$AAu?$AAn?$AA?$AA@ 10002688     LIBCMT:nlsdata2.obj
 0001:00001690       ??_C@_17PNNKMEED@?$AAM?$AAa?$AAy?$AA?$AA@ 10002690     LIBCMT:nlsdata2.obj
 0001:00001698       ??_C@_17LFPOIHDD@?$AAA?$AAp?$AAr?$AA?$AA@ 10002698     LIBCMT:nlsdata2.obj
 0001:000016a0       ??_C@_17CKNLEDEC@?$AAM?$AAa?$AAr?$AA?$AA@ 100026a0     LIBCMT:nlsdata2.obj
 0001:000016a8       ??_C@_17LMDJEKJN@?$AAF?$AAe?$AAb?$AA?$AA@ 100026a8     LIBCMT:nlsdata2.obj
 0001:000016b0       ??_C@_17DKNBKCHM@?$AAJ?$AAa?$AAn?$AA?$AA@ 100026b0     LIBCMT:nlsdata2.obj
 0001:000016b8       ??_C@_1BC@ENMNNPAJ@?$AAS?$AAa?$AAt?$AAu?$AAr?$AAd?$AAa?$AAy?$AA?$AA@ 100026b8     LIBCMT:nlsdata2.obj
 0001:000016cc       ??_C@_1O@PDICJHAG@?$AAF?$AAr?$AAi?$AAd?$AAa?$AAy?$AA?$AA@ 100026cc     LIBCMT:nlsdata2.obj
 0001:000016dc       ??_C@_1BC@HHMNLIHE@?$AAT?$AAh?$AAu?$AAr?$AAs?$AAd?$AAa?$AAy?$AA?$AA@ 100026dc     LIBCMT:nlsdata2.obj
 0001:000016f0       ??_C@_1BE@EBOGMDOH@?$AAW?$AAe?$AAd?$AAn?$AAe?$AAs?$AAd?$AAa?$AAy?$AA?$AA@ 100026f0     LIBCMT:nlsdata2.obj
 0001:00001704       ??_C@_1BA@ENFBFFEK@?$AAT?$AAu?$AAe?$AAs?$AAd?$AAa?$AAy?$AA?$AA@ 10002704     LIBCMT:nlsdata2.obj
 0001:00001714       ??_C@_1O@MMNBFLIA@?$AAM?$AAo?$AAn?$AAd?$AAa?$AAy?$AA?$AA@ 10002714     LIBCMT:nlsdata2.obj
 0001:00001724       ??_C@_1O@IHNHDHPB@?$AAS?$AAu?$AAn?$AAd?$AAa?$AAy?$AA?$AA@ 10002724     LIBCMT:nlsdata2.obj
 0001:00001734       ??_C@_17GGIBDPIH@?$AAS?$AAa?$AAt?$AA?$AA@ 10002734     LIBCMT:nlsdata2.obj
 0001:0000173c       ??_C@_17HFOLPPLP@?$AAF?$AAr?$AAi?$AA?$AA@ 1000273c     LIBCMT:nlsdata2.obj
 0001:00001744       ??_C@_17PDPHAADD@?$AAT?$AAh?$AAu?$AA?$AA@ 10002744     LIBCMT:nlsdata2.obj
 0001:0000174c       ??_C@_17CJEDCEPE@?$AAW?$AAe?$AAd?$AA?$AA@ 1000274c     LIBCMT:nlsdata2.obj
 0001:00001754       ??_C@_17BMKGEGOJ@?$AAT?$AAu?$AAe?$AA?$AA@ 10002754     LIBCMT:nlsdata2.obj
 0001:0000175c       ??_C@_17KBOMKBF@?$AAM?$AAo?$AAn?$AA?$AA@ 1000275c     LIBCMT:nlsdata2.obj
 0001:00001764       ??_C@_17MBGCMIPB@?$AAS?$AAu?$AAn?$AA?$AA@ 10002764     LIBCMT:nlsdata2.obj
 0001:0000176c       ??_C@_08JCCMCCIL@HH?3mm?3ss?$AA@ 1000276c     LIBCMT:nlsdata2.obj
 0001:00001778       ??_C@_0BE@CKGJFCPC@dddd?0?5MMMM?5dd?0?5yyyy?$AA@ 10002778     LIBCMT:nlsdata2.obj
 0001:0000178c       ??_C@_08BPBNCDIB@MM?1dd?1yy?$AA@ 1000278c     LIBCMT:nlsdata2.obj
 0001:00001798       ??_C@_02CJNFDJBF@PM?$AA@   10002798     LIBCMT:nlsdata2.obj
 0001:0000179c       ??_C@_02DEDBPAFC@AM?$AA@   1000279c     LIBCMT:nlsdata2.obj
 0001:000017a0       ??_C@_08EDHMEBNP@December?$AA@ 100027a0     LIBCMT:nlsdata2.obj
 0001:000017ac       ??_C@_08HCHEGEOA@November?$AA@ 100027ac     LIBCMT:nlsdata2.obj
 0001:000017b8       ??_C@_07JJNFCEND@October?$AA@ 100027b8     LIBCMT:nlsdata2.obj
 0001:000017c0       ??_C@_09BHHEALKD@September?$AA@ 100027c0     LIBCMT:nlsdata2.obj
 0001:000017cc       ??_C@_06LBBHFDDG@August?$AA@ 100027cc     LIBCMT:nlsdata2.obj
 0001:000017d4       ??_C@_04MIEPOIFP@July?$AA@ 100027d4     LIBCMT:nlsdata2.obj
 0001:000017dc       ??_C@_04CNLMGBGM@June?$AA@ 100027dc     LIBCMT:nlsdata2.obj
 0001:000017e4       ??_C@_05DMJDNLEJ@April?$AA@ 100027e4     LIBCMT:nlsdata2.obj
 0001:000017ec       ??_C@_05HPCKOFNC@March?$AA@ 100027ec     LIBCMT:nlsdata2.obj
 0001:000017f4       ??_C@_08GNJGEPFN@February?$AA@ 100027f4     LIBCMT:nlsdata2.obj
 0001:00001800       ??_C@_07CGJPFGJA@January?$AA@ 10002800     LIBCMT:nlsdata2.obj
 0001:00001808       ??_C@_03MKABNOCG@Dec?$AA@  10002808     LIBCMT:nlsdata2.obj
 0001:0000180c       ??_C@_03JPJOFNIA@Nov?$AA@  1000280c     LIBCMT:nlsdata2.obj
 0001:00001810       ??_C@_03BMAOKBAD@Oct?$AA@  10002810     LIBCMT:nlsdata2.obj
 0001:00001814       ??_C@_03GGCAPAJC@Sep?$AA@  10002814     LIBCMT:nlsdata2.obj
 0001:00001818       ??_C@_03IFJFEIGA@Aug?$AA@  10002818     LIBCMT:nlsdata2.obj
 0001:0000181c       ??_C@_03LBGABGKK@Jul?$AA@  1000281c     LIBCMT:nlsdata2.obj
 0001:00001820       ??_C@_03IDFGHECI@Jun?$AA@  10002820     LIBCMT:nlsdata2.obj
 0001:00001824       ??_C@_03CNMDKL@May?$AA@    10002824     LIBCMT:nlsdata2.obj
 0001:00001828       ??_C@_03LEOLGMJP@Apr?$AA@  10002828     LIBCMT:nlsdata2.obj
 0001:0000182c       ??_C@_03ODNJBKGA@Mar?$AA@  1000282c     LIBCMT:nlsdata2.obj
 0001:00001830       ??_C@_03HJBDCHOM@Feb?$AA@  10002830     LIBCMT:nlsdata2.obj
 0001:00001834       ??_C@_03JIHJHPIE@Jan?$AA@  10002834     LIBCMT:nlsdata2.obj
 0001:00001838       ??_C@_08INBOOONO@Saturday?$AA@ 10002838     LIBCMT:nlsdata2.obj
 0001:00001844       ??_C@_06JECMNKMI@Friday?$AA@ 10002844     LIBCMT:nlsdata2.obj
 0001:0000184c       ??_C@_08HACCIKIA@Thursday?$AA@ 1000284c     LIBCMT:nlsdata2.obj
 0001:00001858       ??_C@_09DLIGFAKA@Wednesday?$AA@ 10002858     LIBCMT:nlsdata2.obj
 0001:00001864       ??_C@_07BAAGCFCM@Tuesday?$AA@ 10002864     LIBCMT:nlsdata2.obj
 0001:0000186c       ??_C@_06JLEDEDGH@Monday?$AA@ 1000286c     LIBCMT:nlsdata2.obj
 0001:00001874       ??_C@_06OOPIFAJ@Sunday?$AA@ 10002874     LIBCMT:nlsdata2.obj
 0001:0000187c       ??_C@_03FEFJNEK@Sat?$AA@   1000287c     LIBCMT:nlsdata2.obj
 0001:00001880       ??_C@_03IDIOELNC@Fri?$AA@  10002880     LIBCMT:nlsdata2.obj
 0001:00001884       ??_C@_03IOFIKPDN@Thu?$AA@  10002884     LIBCMT:nlsdata2.obj
 0001:00001888       ??_C@_03MHOMLAJA@Wed?$AA@  10002888     LIBCMT:nlsdata2.obj
 0001:0000188c       ??_C@_03NAGEINEP@Tue?$AA@  1000288c     LIBCMT:nlsdata2.obj
 0001:00001890       ??_C@_03PDAGKDH@Mon?$AA@   10002890     LIBCMT:nlsdata2.obj
 0001:00001894       ??_C@_03KOEHGMDN@Sun?$AA@  10002894     LIBCMT:nlsdata2.obj
 0001:00001898       ??_C@_0BI@DFKBFLJE@GetProcessWindowStation?$AA@ 10002898     LIBCMT:crtmboxw.obj
 0001:000018b0       ??_C@_0BK@DEKFELLI@GetUserObjectInformationW?$AA@ 100028b0     LIBCMT:crtmboxw.obj
 0001:000018cc       ??_C@_0BD@HHGDFDBJ@GetLastActivePopup?$AA@ 100028cc     LIBCMT:crtmboxw.obj
 0001:000018e0       ??_C@_0BA@HNOPNCHB@GetActiveWindow?$AA@ 100028e0     LIBCMT:crtmboxw.obj
 0001:000018f0       ??_C@_0M@DLDCCGNP@MessageBoxW?$AA@ 100028f0     LIBCMT:crtmboxw.obj
 0001:000018fc       ??_C@_1BG@GOEBHBDC@?$AAU?$AAS?$AAE?$AAR?$AA3?$AA2?$AA?4?$AAD?$AAL?$AAL?$AA?$AA@ 100028fc     LIBCMT:crtmboxw.obj
 0001:00001918       ___newctype                10002918     LIBCMT:ctype.obj
 0001:00001c18       __wctype                   10002c18     LIBCMT:ctype.obj
 0001:00001e20       ___newclmap                10002e20     LIBCMT:ctype.obj
 0001:00001fa0       ___newcumap                10002fa0     LIBCMT:ctype.obj
 0001:00002128       __load_config_used         10003128     LIBCMT:loadcfg.obj
 0001:00002170       ___safe_se_handler_table   10003170     <linker-defined>
 0001:0000217c       ___rtc_iaa                 1000317c     LIBCMT:_initsect_.obj
 0001:00002180       ___rtc_izz                 10003180     LIBCMT:_initsect_.obj
 0001:00002184       ___rtc_taa                 10003184     LIBCMT:_initsect_.obj
 0001:00002188       ___rtc_tzz                 10003188     LIBCMT:_initsect_.obj
 0001:00002190       __alloca_probe             10003190     chkstk.obj
 0001:00002190       __chkstk                   10003190 f   chkstk.obj
 0001:000021c0       _DlgProc@16                100031c0 f   luaplug.obj
 0001:00002250       _DllMain@12                10003250 f   luaplug.obj
 0001:00002300       _luaopen_luaplug           10003300 f   luaplug.obj
 0001:000023a0       _GetLuaState               100033a0 f   luaplug.obj
 0001:000023b0       _GetGlobalInfoW@4          100033b0 f   luaplug.obj
 0001:00002440       _SetStartupInfoW@4         10003440 f   luaplug.obj
 0001:00002510       _GetPluginInfoW@4          10003510 f   luaplug.obj
 0001:00002530       _ProcessSynchroEventW@4    10003530 f   luaplug.obj
 0001:00002560       _GetMinFarVersionW@0       10003560 f   luaplug.obj
 0001:00002670       _OpenW@4                   10003670 f   luaplug.obj
 0001:000026f0       _ExitFARW@4                100036f0 f   luaplug.obj
 0001:00002730       _ConfigureW@4              10003730 f   luaplug.obj
 0001:00002760       _ProcessEditorInputW@4     10003760 f   luaplug.obj
 0001:00002790       _ProcessEditorEventW@4     10003790 f   luaplug.obj
 0001:000027c0       _ProcessViewerEventW@4     100037c0 f   luaplug.obj
 0001:000027f0       _ProcessDialogEventW@4     100037f0 f   luaplug.obj
 0001:00002890       _EncodePointerWrapper@4    10003890 f   vc_crt_fix_impl.obj
 0001:000028e0       _DecodePointerWrapper@4    100038e0 f   vc_crt_fix_impl.obj
 0001:00002930       _GetModuleHandleExWWrapper@12 10003930 f   vc_crt_fix_impl.obj
 0001:00002974       _luaL_error                10003974 f   lua51:lua51.dll
 0001:0000297a       _lua_sethook               1000397a f   lua51:lua51.dll
 0001:00002980       _lua_close                 10003980 f   lua51:lua51.dll
 0001:00002986       _luaL_newstate             10003986 f   lua51:lua51.dll
 0001:0000298c       _luaL_ref                  1000398c f   lua51:lua51.dll
 0001:00002992       _lua_newuserdata           10003992 f   lua51:lua51.dll
 0001:00002998       _lua_setfield              10003998 f   lua51:lua51.dll
 0001:0000299e       _lua_pushcclosure          1000399e f   lua51:lua51.dll
 0001:000029a4       _lua_settop                100039a4 f   lua51:lua51.dll
 0001:000029aa       _lua_pushboolean           100039aa f   lua51:lua51.dll
 0001:000029b0       _lua_toboolean             100039b0 f   lua51:lua51.dll
 0001:000029b6       _lua_getfield              100039b6 f   lua51:lua51.dll
 0001:000029bc       __initp_misc_winsig        100039bc f   LIBCMT:winsig.obj
 0001:00002aad       ___get_sigabrt             10003aad f   LIBCMT:winsig.obj
 0001:00002aba       _signal                    10003aba f   LIBCMT:winsig.obj
 0001:00002cfa       _raise                     10003cfa f   LIBCMT:winsig.obj
 0001:00002e9d       _wcsrchr                   10003e9d f   LIBCMT:wcsrchr.obj
 0001:00002ecb       __CRT_INIT@12              10003ecb f   LIBCMT:dllcrt0.obj
 0001:00003125       __DllMainCRTStartup@12     10004125 f   LIBCMT:dllcrt0.obj
 0001:00003148       __mtinitlocks              10004148 f   LIBCMT:mlock.obj
 0001:00003192       __mtdeletelocks            10004192 f   LIBCMT:mlock.obj
 0001:000031e9       __unlock                   100041e9 f   LIBCMT:mlock.obj
 0001:00003200       __mtinitlocknum            10004200 f   LIBCMT:mlock.obj
 0001:000032c2       __lock                     100042c2 f   LIBCMT:mlock.obj
 0001:000032f5       __encoded_null             100042f5 f   LIBCMT:tidtable.obj
 0001:000032fe       ___crtTlsAlloc@4           100042fe f   LIBCMT:tidtable.obj
 0001:00003307       ___set_flsgetvalue         10004307 f   LIBCMT:tidtable.obj
 0001:0000333b       __mtterm                   1000433b f   LIBCMT:tidtable.obj
 0001:00003378       __initptd                  10004378 f   LIBCMT:tidtable.obj
 0001:0000342c       __getptd_noexit            1000442c f   LIBCMT:tidtable.obj
 0001:000034a5       __getptd                   100044a5 f   LIBCMT:tidtable.obj
 0001:000034bf       __freefls@4                100044bf f   LIBCMT:tidtable.obj
 0001:000035ee       __freeptd                  100045ee f   LIBCMT:tidtable.obj
 0001:0000365c       __mtinit                   1000465c f   LIBCMT:tidtable.obj
 0001:000037e0       __SEH_prolog4              100047e0 f   LIBCMT:sehprolg4.obj
 0001:00003825       __SEH_epilog4              10004825 f   LIBCMT:sehprolg4.obj
 0001:00003840       __except_handler4          10004840 f   LIBCMT:chandler4.obj
 0001:000039cf       __XcptFilter               100049cf f   LIBCMT:winxfltr.obj
 0001:00003b19       ___CppXcptFilter           10004b19 f   LIBCMT:winxfltr.obj
 0001:00003b39       __initp_misc_invarg        10004b39 f   LIBCMT:invarg.obj
 0001:00003b48       __call_reportfault         10004b48 f   LIBCMT:invarg.obj
 0001:00003c71       __invoke_watson            10004c71 f   LIBCMT:invarg.obj
 0001:00003c96       __invalid_parameter        10004c96 f   LIBCMT:invarg.obj
 0001:00003cc3       __invalid_parameter_noinfo 10004cc3 f   LIBCMT:invarg.obj
 0001:00003cd3       __get_errno_from_oserr     10004cd3 f   LIBCMT:dosmap.obj
 0001:00003d15       __errno                    10004d15 f   LIBCMT:dosmap.obj
 0001:00003d28       ___doserrno                10004d28 f   LIBCMT:dosmap.obj
 0001:00003d40       _memcpy                    10004d40 f   LIBCMT:memcpy.obj
 0001:000040a1       __malloc_crt               100050a1 f   LIBCMT:crtheap.obj
 0001:000040e6       __calloc_crt               100050e6 f   LIBCMT:crtheap.obj
 0001:00004132       __realloc_crt              10005132 f   LIBCMT:crtheap.obj
 0001:00004180       ___crtCorExitProcess       10005180 f   LIBCMT:crt0dat.obj
 0001:000041ab       ___crtExitProcess          100051ab f   LIBCMT:crt0dat.obj
 0001:000041c3       __lockexit                 100051c3 f   LIBCMT:crt0dat.obj
 0001:000041cc       __unlockexit               100051cc f   LIBCMT:crt0dat.obj
 0001:000041d5       __init_pointers            100051d5 f   LIBCMT:crt0dat.obj
 0001:00004208       __initterm_e               10005208 f   LIBCMT:crt0dat.obj
 0001:0000422c       __cinit                    1000522c f   LIBCMT:crt0dat.obj
 0001:00004403       __exit                     10005403 f   LIBCMT:crt0dat.obj
 0001:00004419       __cexit                    10005419 f   LIBCMT:crt0dat.obj
 0001:00004428       __amsg_exit                10005428 f   LIBCMT:crt0dat.obj
 0001:00004446       _free                      10005446 f   LIBCMT:free.obj
 0001:00004480       __ioinit                   10005480 f   LIBCMT:ioinit.obj
 0001:000046c5       __ioterm                   100056c5 f   LIBCMT:ioinit.obj
 0001:00004718       __setenvp                  10005718 f   LIBCMT:stdenvp.obj
 0001:0000498e       __setargv                  1000598e f   LIBCMT:stdargv.obj
 0001:00004a49       ___crtGetEnvironmentStringsA 10005a49 f   LIBCMT:a_env.obj
 0001:00004ae0       __RTC_Initialize           10005ae0 f   LIBCMT:_initsect_.obj
 0001:00004b06       __RTC_Terminate            10005b06 f   LIBCMT:_initsect_.obj
 0001:00004b2c       __heap_init                10005b2c f   LIBCMT:heapinit.obj
 0001:00004b4a       __heap_term                10005b4a f   LIBCMT:heapinit.obj
 0001:00004b5e       ___security_init_cookie    10005b5e f   LIBCMT:gs_support.obj
 0001:00004bf9       __GET_RTERRMSG             10005bf9 f   LIBCMT:crt0msg.obj
 0001:00004c1f       __NMSG_WRITE               10005c1f f   LIBCMT:crt0msg.obj
 0001:00004dce       __FF_MSGBANNER             10005dce f   LIBCMT:crt0msg.obj
 0001:00004e07       ___addlocaleref            10005e07 f   LIBCMT:localref.obj
 0001:00004e96       ___removelocaleref         10005e96 f   LIBCMT:localref.obj
 0001:00004f2f       ___freetlocinfo            10005f2f f   LIBCMT:localref.obj
 0001:0000507a       __updatetlocinfoEx_nolock  1000607a f   LIBCMT:localref.obj
 0001:000050c7       ___updatetlocinfo          100060c7 f   LIBCMT:localref.obj
 0001:00005363       ___updatetmbcinfo          10006363 f   LIBCMT:mbctype.obj
 0001:00005407       ??0_LocaleUpdate@@QAE@PAUlocaleinfo_struct@@@Z 10006407 f i LIBCMT:mbctype.obj
 0001:0000550a       __setmbcp_nolock           1000650a f   LIBCMT:mbctype.obj
 0001:000056f3       __setmbcp                  100066f3 f   LIBCMT:mbctype.obj
 0001:0000588d       ___initmbctable            1000688d f   LIBCMT:mbctype.obj
 0001:000058ab       @__security_check_cookie@4 100068ab f   LIBCMT:secchk.obj
 0001:000058c0       __local_unwind4            100068c0 f   LIBCMT:exsup4.obj
 0001:00005996       __seh_longjmp_unwind4@4    10006996 f   LIBCMT:exsup4.obj
 0001:000059b2       @_EH4_CallFilterFunc@8     100069b2 f   LIBCMT:exsup4.obj
 0001:000059c9       @_EH4_TransferToHandler@8  100069c9 f   LIBCMT:exsup4.obj
 0001:000059e2       @_EH4_GlobalUnwind2@8      100069e2 f   LIBCMT:exsup4.obj
 0001:000059fb       @_EH4_LocalUnwind@16       100069fb f   LIBCMT:exsup4.obj
 0001:00005a20       __ValidateImageBase        10006a20 f   LIBCMT:pesect.obj
 0001:00005a60       __FindPESection            10006a60 f   LIBCMT:pesect.obj
 0001:00005ab0       __IsNonwritableInCurrentImage 10006ab0 f   LIBCMT:pesect.obj
 0001:00005b6c       __crt_debugger_hook        10006b6c f   LIBCMT:dbghook.obj
 0001:00005b80       _memset                    10006b80 f   LIBCMT:memset.obj
 0001:00005bfa       __VEC_memcpy               10006bfa f   LIBCMT:p4_memcpy.obj
 0001:00005cfd       ___sse2_available_init     10006cfd f   LIBCMT:cpu_disp.obj
 0001:00005d0d       _malloc                    10006d0d f   LIBCMT:malloc.obj
 0001:00005da1       __calloc_impl              10006da1 f   LIBCMT:calloc_impl.obj
 0001:00005e23       _realloc                   10006e23 f   LIBCMT:realloc.obj
 0001:00005ed0       ?terminate@@YAXXZ          10006ed0 f   LIBCMT:hooks.obj
 0001:00005f09       __initp_eh_hooks           10006f09 f   LIBCMT:hooks.obj
 0001:00005f1a       __initp_misc_rand_s        10006f1a f   LIBCMT:rand_s.obj
 0001:00005f29       __initp_misc_purevirt      10006f29 f   LIBCMT:inithelp.obj
 0001:00005f38       __initp_heap_handler       10006f38 f   LIBCMT:handler.obj
 0001:00005f47       __callnewh                 10006f47 f   LIBCMT:handler.obj
 0001:00006028       ___onexitinit              10007028 f   LIBCMT:onexit.obj
 0001:00006059       __onexit                   10007059 f   LIBCMT:onexit.obj
 0001:00006095       _atexit                    10007095 f   LIBCMT:onexit.obj
 0001:000060ac       __initp_misc_cfltcvt_tab   100070ac f   LIBCMT:cmiscdat.obj
 0001:000060cf       _strcpy_s                  100070cf f   LIBCMT:strcpy_s.obj
 0001:00006130       _strlen                    10007130 f   LIBCMT:strlen.obj
 0001:0000620e       __ismbblead                1000720e f   LIBCMT:ismbbyte.obj
 0001:00006226       ___crtMessageBoxW          10007226 f   LIBCMT:crtmboxw.obj
 0001:00006392       _wcscat_s                  10007392 f   LIBCMT:wcscat_s.obj
 0001:00006407       _wcsncpy_s                 10007407 f   LIBCMT:wcsncpy_s.obj
 0001:000064d4       _wcslen                    100074d4 f   LIBCMT:wcslen.obj
 0001:000064ef       _wcscpy_s                  100074ef f   LIBCMT:wcscpy_s.obj
 0001:00006552       __set_error_mode           10007552 f   LIBCMT:errmode.obj
 0001:00006591       ___free_lc_time            10007591 f   LIBCMT:inittime.obj
 0001:00006908       ___free_lconv_num          10007908 f   LIBCMT:initnum.obj
 0001:00006971       ___free_lconv_mon          10007971 f   LIBCMT:initmon.obj
 0001:00006a6f       __freea                    10007a6f f i LIBCMT:a_map.obj
 0001:00006c76       ___crtLCMapStringA         10007c76 f   LIBCMT:a_map.obj
 0001:00006da3       ___crtGetStringTypeA       10007da3 f   LIBCMT:a_str.obj
 0001:00006de3       ___report_gsfailure        10007de3 f   LIBCMT:gs_report.obj
 0001:00006f00       __global_unwind2           10007f00 f   LIBCMT:exsup.obj
 0001:00006f65       __local_unwind2            10007f65 f   LIBCMT:exsup.obj
 0001:00006fe9       __abnormal_termination     10007fe9 f   LIBCMT:exsup.obj
 0001:0000700c       __NLG_Notify1              1000800c f   LIBCMT:exsup.obj
 0001:00007015       __NLG_Notify               10008015 f   LIBCMT:exsup.obj
 0001:0000702c       __NLG_Dispatch             1000802c     LIBCMT:exsup.obj
 0001:0000702c       __NLG_Dispatch2            1000802c     LIBCMT:exsup.obj
 0001:00007034       __NLG_Call                 10008034 f   LIBCMT:exsup.obj
 0001:00007036       __NLG_Return2              10008036     LIBCMT:exsup.obj
 0001:00007037       __VEC_memzero              10008037 f   LIBCMT:p4_memset.obj
 0001:000070f1       __msize                    100080f1 f   LIBCMT:msize.obj
 0001:00007124       _abort                     10008124 f   LIBCMT:abort.obj
 0001:00007157       __fptrap                   10008157 f   LIBCMT:crt0fp.obj
 0001:00007160       __alloca_probe_16          10008160 f   LIBCMT:alloca16.obj
 0001:00007176       __alloca_probe_8           10008176     LIBCMT:alloca16.obj
 0001:0000718c       _RtlUnwind@16              1000818c f   kernel32:KERNEL32.dll
 0001:00007384       __IMPORT_DESCRIPTOR_KERNEL32 10008384     kernel32:KERNEL32.dll
 0001:00007398       __IMPORT_DESCRIPTOR_lua51  10008398     lua51:lua51.dll
 0001:000073ac       __IMPORT_DESCRIPTOR_luafar3 100083ac     luafar3:luafar3.dll
 0001:000073c0       __NULL_IMPORT_DESCRIPTOR   100083c0     kernel32:KERNEL32.dll
 0002:00000000       _PluginData                10009000     luaplug.obj
 0002:00000150       ___flsindex                10009150     LIBCMT:tidtable.obj
 0002:00000154       ___getvalueindex           10009154     LIBCMT:tidtable.obj
 0002:000002d0       ___badioinfo               100092d0     LIBCMT:ioinit.obj
 0002:00000310       ___clocalestr              10009310     LIBCMT:nlsdata2.obj
 0002:00000318       ___lc_time_c               10009318     LIBCMT:nlsdata2.obj
 0002:00000480       ___initiallocinfo          10009480     LIBCMT:nlsdata2.obj
 0002:00000558       ___ptlocinfo               10009558     LIBCMT:nlsdata2.obj
 0002:00000560       ___initialmbcinfo          10009560     LIBCMT:mbctype.obj
 0002:00000780       __mbctype                  10009780     LIBCMT:mbctype.obj
 0002:00000888       __mbcasemap                10009888     LIBCMT:mbctype.obj
 0002:00000988       ___ptmbcinfo               10009988     LIBCMT:mbctype.obj
 0002:00000a80       ___security_cookie         10009a80     LIBCMT:gs_cookie.obj
 0002:00000a84       ___security_cookie_complement 10009a84     LIBCMT:gs_cookie.obj
 0002:00000a90       __cfltcvt_tab              10009a90     LIBCMT:cmiscdat.obj
 0002:00000ac0       ___lconv_static_decimal    10009ac0     LIBCMT:lconv.obj
 0002:00000ac4       ___lconv_static_W_decimal  10009ac4     LIBCMT:lconv.obj
 0002:00000ac8       ___lconv_c                 10009ac8     LIBCMT:lconv.obj
 0002:00000b18       ___lconv                   10009b18     LIBCMT:lconv.obj
 0002:00000b1c       ___globallocalestatus      10009b1c     LIBCMT:glstatus.obj
 0002:00000b20       __pctype                   10009b20     LIBCMT:ctype.obj
 0002:00000b24       __pwctype                  10009b24     LIBCMT:ctype.obj
 0002:00000b30       __NLG_Destination          10009b30     LIBCMT:exsup.obj
 0002:00000b40       ___abort_behavior          10009b40     LIBCMT:abort.obj
 0002:00000b60       _Init1_Done                10009b60     luaplug.obj
 0002:00000b64       _Init2_Done                10009b64     luaplug.obj
 0002:00000b9c       __aenvptr                  10009b9c     LIBCMT:dllcrt0.obj
 0002:00000ba0       __wenvptr                  10009ba0     LIBCMT:dllcrt0.obj
 0002:00000ba4       ___error_mode              10009ba4     LIBCMT:dllcrt0.obj
 0002:00000ba8       ___app_type                10009ba8     LIBCMT:dllcrt0.obj
 0002:00000d00       _gpFlsAlloc                10009d00     LIBCMT:tidtable.obj
 0002:00000d04       _gpFlsGetValue             10009d04     LIBCMT:tidtable.obj
 0002:00000d08       _gpFlsSetValue             10009d08     LIBCMT:tidtable.obj
 0002:00000d0c       _gpFlsFree                 10009d0c     LIBCMT:tidtable.obj
 0002:00000d10       ___pInvalidArgHandler      10009d10     LIBCMT:invarg.obj
 0002:00000d14       __maxwait                  10009d14     LIBCMT:crtheap.obj
 0002:00000d18       __umaskval                 10009d18     LIBCMT:crt0dat.obj
 0002:00000d1c       ___argc                    10009d1c     LIBCMT:crt0dat.obj
 0002:00000d20       ___argv                    10009d20     LIBCMT:crt0dat.obj
 0002:00000d24       ___wargv                   10009d24     LIBCMT:crt0dat.obj
 0002:00000d28       __environ                  10009d28     LIBCMT:crt0dat.obj
 0002:00000d2c       ___initenv                 10009d2c     LIBCMT:crt0dat.obj
 0002:00000d30       __wenviron                 10009d30     LIBCMT:crt0dat.obj
 0002:00000d34       ___winitenv                10009d34     LIBCMT:crt0dat.obj
 0002:00000d38       __pgmptr                   10009d38     LIBCMT:crt0dat.obj
 0002:00000d3c       __wpgmptr                  10009d3c     LIBCMT:crt0dat.obj
 0002:00000d40       __exitflag                 10009d40     LIBCMT:crt0dat.obj
 0002:00000d44       __C_Termination_Done       10009d44     LIBCMT:crt0dat.obj
 0002:00000d48       __C_Exit_Done              10009d48     LIBCMT:crt0dat.obj
 0002:00000e58       __crtheap                  10009e58     LIBCMT:heapinit.obj
 0002:0000148c       ___mbulinfo                1000a48c     LIBCMT:mbctype.obj
 0002:00001498       ___mbcodepage              1000a498     LIBCMT:mbctype.obj
 0002:0000149c       ___ismbcodepage            1000a49c     LIBCMT:mbctype.obj
 0002:000014a0       ___mblcid                  1000a4a0     LIBCMT:mbctype.obj
 0002:000014a4       ?__pInconsistency@@3P6AXXZA 1000a4a4     LIBCMT:hooks.obj
 0002:000014ac       ___pPurecall               1000a4ac     LIBCMT:inithelp.obj
 0002:000014b0       ?_pnhHeap@@3P6AHI@ZA       1000a4b0     LIBCMT:handler.obj
 0002:000014c8       ___lconv_static_null       1000a4c8     LIBCMT:lconv.obj
 0002:000014cc       ___lconv_static_W_null     1000a4cc     LIBCMT:lconv.obj
 0002:000017f4       __newmode                  1000a7f4     LIBCMT:_newmode.obj
 0002:00001800       _PluginDir                 1000a800     <common>
 0002:00001c00       _FindFileSection           1000ac00     <common>
 0002:00001c20       _Info                      1000ac20     <common>
 0002:00001cc0       _PluginName                1000acc0     <common>
 0002:000020c0       _LS                        1000b0c0     <common>
 0002:000020d0       _PluginId                  1000b0d0     <common>
 0002:000020e0       _FSF                       1000b0e0     <common>
 0002:0000219c       ___sse2_available          1000b19c     <common>
 0002:000021a0       __debugger_hook_dummy      1000b1a0     <common>
 0002:000021a4       __nhandle                  1000b1a4     <common>
 0002:000021c0       ___pioinfo                 1000b1c0     <common>
 0002:000022c0       ___env_initialized         1000b2c0     <common>
 0002:000022c4       ___onexitend               1000b2c4     <common>
 0002:000022c8       ___onexitbegin             1000b2c8     <common>
 0002:000022cc       ___mbctype_initialized     1000b2cc     <common>
 0002:000022d0       __FPinit                   1000b2d0     <common>
 0002:000022d4       ___dyn_tls_init_callback   1000b2d4     <common>
 0002:000022d8       __pDestructExceptionObject 1000b2d8     <common>
 0002:000022dc       __acmdln                   1000b2dc     <common>

 entry point at        0001:00003125

 Static symbols

 0001:000021f0       _lstop                     100031f0 f   luaplug.obj
 0001:00002220       _laction                   10003220 f   luaplug.obj
 0001:00002350       _InitLuaState2             10003350 f   luaplug.obj
 0001:00002570       _RecreateLuaState          10003570 f   luaplug.obj
 0001:00002840       ?EncodePointer@implementation@?1??EncodePointerWrapper@@9@4@SGPAXPAX@Z 10003840 f   vc_crt_fix_impl.obj
 0001:00002840       ?DecodePointer@implementation@?1??DecodePointerWrapper@@9@4@SGPAXPAX@Z 10003840 f   vc_crt_fix_impl.obj
 0001:00002850       ?GetModuleHandleExW@implementation@?1??GetModuleHandleExWWrapper@@9@12@SGHKPB_WPAPAUHINSTANCE__@@@Z 10003850 f   vc_crt_fix_impl.obj
 0001:000029da       _ctrlevent_capture@4       100039da f   LIBCMT:winsig.obj
 0001:00002a76       _siglookup                 10003a76 f   LIBCMT:winsig.obj
 0001:0000302f       ___DllMainCRTStartup       1000402f f   LIBCMT:dllcrt0.obj
 0001:000042c3       _doexit                    100052c3 f   LIBCMT:crt0dat.obj
 0001:000047f4       _parse_cmdline             100057f4 f   LIBCMT:stdargv.obj
 0001:00005140       ?CPtoLCID@@YAHH@Z          10006140 f   LIBCMT:mbctype.obj
 0001:0000516f       ?setSBCS@@YAXPAUthreadmbcinfostruct@@@Z 1000616f f   LIBCMT:mbctype.obj
 0001:000051d3       ?setSBUpLow@@YAXPAUthreadmbcinfostruct@@@Z 100061d3 f   LIBCMT:mbctype.obj
 0001:0000548e       ?getSystemCP@@YAHH@Z       1000648e f   LIBCMT:mbctype.obj
 0001:00005950       __unwind_handler4          10006950 f   LIBCMT:exsup4.obj
 0001:00005f72       __onexit_nolock            10006f72 f   LIBCMT:onexit.obj
 0001:000061bb       ?x_ismbbtype_l@@YAHPAUlocaleinfo_struct@@IHH@Z 100071bb f   LIBCMT:ismbbyte.obj
 0001:00006a8f       ?__crtLCMapStringA_stat@@YAHPAUlocaleinfo_struct@@KKPBDHPADHHH@Z 10007a8f f   LIBCMT:a_map.obj
 0001:00006cbc       ?__crtGetStringTypeA_stat@@YAHPAUlocaleinfo_struct@@KPBDHPAGHHH@Z 10007cbc f   LIBCMT:a_str.obj
 0001:00006f20       __unwind_handler           10007f20 f   LIBCMT:exsup.obj
